******************************************************************************
                  TI ARM Linker PC v5.1.5                      
******************************************************************************
>> Linked Mon Mar 30 09:25:19 2015

OUTPUT FILE NAME:   <EDCU_TMS570LS1227.pi.out>
ENTRY POINT SYMBOL: "_c_int00"  address: 00010584


MEMORY CONFIGURATION

         name            origin    length      used     unused   attr    fill
----------------------  --------  ---------  --------  --------  ----  --------
  VECTORS               00000000   00000020  00000020  00000000     X
  FLASH0                00000020   0013ffe0  000122dc  0012dd04  R  X
  STACKS                08000000   00001500  00000000  00001500  RW  
  RAM                   08001500   0002eb00  00002dd0  0002bd30  RW  


SEGMENT ALLOCATION MAP

run origin  load origin   length   init length attrs members
----------  ----------- ---------- ----------- ----- -------
00000000    00000000    00012300   00012300    r-x
  00000000    00000000    00000020   00000020    r-x .intvecs
  00000020    00000020    000119f4   000119f4    r-x .text
  00011a14    00011a14    00000610   00000610    r-- .const
  00012028    00012028    000002d8   000002d8    r-- .cinit
08001500    08001500    00002dd0   00000000    rw-
  08001500    08001500    000027f0   00000000    rw- .bss
  08003cf0    08003cf0    000005e0   00000000    rw- .data


SECTION ALLOCATION MAP

 output                                  attributes/
section   page    origin      length       input sections
--------  ----  ----------  ----------   ----------------
.intvecs   0    00000000    00000020     
                  00000000    00000020     sys_intvecs.obj (.intvecs)

.text      0    00000020    000119f4     
                  00000020    00002ccc     sys_selftest.obj (.text)
                  00002cec    00002394     etpwm.obj (.text)
                  00005080    00001f10     dlsw_motorc.obj (.text)
                  00006f90    000011f4     spi.obj (.text)
                  00008184    00000b48     can.obj (.text)
                  00008ccc    00000b2c     system.obj (.text)
                  000097f8    00000afc     adc.obj (.text)
                  0000a2f4    00000a50     sys_vim.obj (.text)
                  0000ad44    00000930     pinmux.obj (.text)
                  0000b674    000008f4     het.obj (.text)
                  0000bf68    000008d0     ecap.obj (.text)
                  0000c838    00000858     drv_spi.obj (.text)
                  0000d090    00000724     dlsw_io.obj (.text)
                  0000d7b4    00000648     lin.obj (.text)
                  0000ddfc    00000634     esm.obj (.text)
                  0000e430    00000634     rti.obj (.text)
                  0000ea64    000005f0     sci.obj (.text)
                  0000f054    00000484     gio.obj (.text)
                  0000f4d8    00000460     dlsw_timer.obj (.text)
                  0000f938    000003c4     sys_core.obj (.text)
                  0000fcfc    00000300     sys_mpu.obj (.text)
                  0000fffc    000002dc     sys_vim.obj (.text:retain)
                  000102d8    000002ac     spi.obj (.text:retain)
                  00010584    00000270     sys_startup.obj (.text:retain)
                  000107f4    0000021c     sys_main.obj (.text)
                  00010a10    000001c8     notification.obj (.text)
                  00010bd8    00000198     ecap.obj (.text:retain)
                  00010d70    0000016c     pi.obj (.text)
                  00010edc    00000158     esm.obj (.text:retain)
                  00011034    00000114     sys_pmu.obj (.text)
                  00011148    000000e8     dabort.obj (.text)
                  00011230    000000e0     dlsw_draw.obj (.text)
                  00011310    000000c0     drv_public.obj (.text)
                  000113d0    000000ac     dlsw_adc.obj (.text)
                  0001147c    000000a4     adc.obj (.text:retain)
                  00011520    000000a0     drv.obj (.text)
                  000115c0    0000009c     rtsv7R4_T_be_v3D16_eabi.lib : memcpy_t2.obj (.text)
                  0001165c    00000098     gio.obj (.text:retain)
                  000116f4    00000094     rti.obj (.text:retain)
                  00011788    00000094     rtsv7R4_T_be_v3D16_eabi.lib : auto_init.obj (.text)
                  0001181c    00000078                                 : memset_t2.obj (.text)
                  00011894    00000060                                 : copy_decompress_rle.obj (.text)
                  000118f4    00000054                                 : u_div32.obj (.text)
                  00011948    00000048                                 : cpy_tbl.obj (.text)
                  00011990    00000044                                 : exit.obj (.text)
                  000119d4    00000014                                 : _lock.obj (.text)
                  000119e8    00000012                                 : copy_zero_init.obj (.text:decompress:ZI)
                  000119fa    0000000e                                 : copy_decompress_none.obj (.text:decompress:none)
                  00011a08    00000006                                 : copy_decompress_rle.obj (.text:decompress:rle24)
                  00011a0e    00000002     --HOLE-- [fill = 0]
                  00011a10    00000004     sys_phantom.obj (.text:retain)

.const     0    00011a14    00000610     
                  00011a14    000003a0     het.obj (.const:het1PROGRAM)
                  00011db4    00000200     sys_vim.obj (.const:s_vim_init)
                  00011fb4    00000030     adc.obj (.const)
                  00011fe4    00000020     can.obj (.const)
                  00012004    00000020     het.obj (.const)

.cinit     0    00012028    000002d8     
                  00012028    000002b1     (.cinit..data.load) [load image, compression = rle]
                  000122d9    00000003     --HOLE-- [fill = 0]
                  000122dc    0000000c     (__TI_handler_table)
                  000122e8    00000008     (.cinit..bss.load) [load image, compression = zero_init]
                  000122f0    00000010     (__TI_cinit_table)

.bss       0    08001500    000027f0     UNINITIALIZED
                  08001500    00001000     sys_main.obj (.bss:draw1)
                  08002500    00001000     sys_main.obj (.bss:draw2)
                  08003500    00000670     sys_main.obj (.bss:drl)
                  08003b70    00000078     spi.obj (.bss:g_spiPacket_t)
                  08003be8    00000050     drv_spi.obj (.bss:ucReceiveBufferArray)
                  08003c38    00000030     sys_main.obj (.bss:daw)
                  08003c68    00000030     drv_spi.obj (.bss:ucSendBufferArray)
                  08003c98    00000028     sci.obj (.bss:g_sciTransfer_t)
                  08003cc0    00000012     (.common:gstSPICmdStatus)
                  08003cd2    0000000c     (.common:stAqctlaInit)
                  08003cde    00000008     (.common:stDeadBandInit)
                  08003ce6    00000004     (.common:dataconfig1_t)
                  08003cea    00000002     --HOLE--
                  08003cec    00000004     (.common:delayval$1)

.data      0    08003cf0    000005e0     UNINITIALIZED
                  08003cf0    00000200     drv_public.obj (.data:crc16_table)
                  08003ef0    00000180     sys_main.obj (.data:mtr)
                  08004070    0000014c     sys_main.obj (.data:tmr)
                  080041bc    000000c4     sys_main.obj (.data:io)
                  08004280    00000029     drv_spi.obj (.data)
                  080042a9    00000003     --HOLE--
                  080042ac    00000014     sys_main.obj (.data)
                  080042c0    00000008     rtsv7R4_T_be_v3D16_eabi.lib : _lock.obj (.data)
                  080042c8    00000008                                 : exit.obj (.data)


LINKER GENERATED COPY TABLES

__TI_cinit_table @ 000122f0 records: 2, size/record: 8, table size: 16
	.data: load addr=00012028, load size=000002b1 bytes, run addr=08003cf0, run size=000005e0 bytes, compression=rle
	.bss: load addr=000122e8, load size=00000008 bytes, run addr=08001500, run size=000027f0 bytes, compression=zero_init


LINKER GENERATED HANDLER TABLE

__TI_handler_table @ 000122dc records: 3, size/record: 4, table size: 12
	index: 0, handler: __TI_zero_init
	index: 1, handler: __TI_decompress_rle24
	index: 2, handler: __TI_decompress_none


GLOBAL SYMBOLS: SORTED ALPHABETICALLY BY Name 

address    name
--------   ----
00011991   C$$EXIT
00006314   CalculatePWMComp
00010948   CapIntSrv
00006654   CheckDirection
00005d04   ClearMtrPrtctCntr
00006b28   ClearSpdToZero
00005d18   ClearSpeedFeedback
0000f900   CnfgrWatchDogRegister
0000604c   CntrlAcrPi
00005d2c   CntrlAsrPi
000056bc   CntrlMotorStartStop
00005678   CntrlMtrProtection
00010d70   CntrlPID
00006b80   CntrlPWMOutput
00005080   DRV_Motor_start
000050b8   DRV_Motor_stop
0000f934   DisableDog
0000f904   DlyLogicTimer
00011230   DrawPicture1ms
00011520   Drv_Init
0000d244   FilterInput00
0000d2bc   FilterInput01
0000d334   FilterInput02
0000d3ac   FilterInput04
0000d424   FilterInput13
0000d49c   FilterInput14
0000d514   FilterMntnPshBttn
00005648   HandleGPTmr2PrdInt
0000e79c   IsdwdKeySequenceCorrect
00005128   PWM_write_CmpA
0000614c   PiAcr
00005e50   PiAsr
00005178   PwmInit
00006a74   ReadCapSignal
0000d6b0   ReadDoorAddress
0000d090   ReadInputSignal
00005b2c   ReadMotorOffsetIdc
000113d0   ReadMotorRawIdc
000050fc   ReloadCapIntOVCnt
0000638c   ResetSpeedTimer
UNDEFED    SHT$$INIT_ARRAY$$Base
UNDEFED    SHT$$INIT_ARRAY$$Limit
0000cbb4   SPI_DataInit
0000cba0   SPI_Process
00007a7c   SpiRxStatus
000079f0   SpiTxStatus
080042bc   T
0000f4d8   Update100msTimer
0000f580   Update10msTimer
0000f628   Update1msTimer
00006904   UpdateCurrent
0000f6a4   UpdateCurrentTime
0000d5d8   UpdateInputSignal
0000f8c0   UpdateMtrRttnTimer
000063d0   UpdateSpeed
000122f0   __TI_CINIT_Base
00012300   __TI_CINIT_Limit
000122dc   __TI_Handler_Table_Base
000122e8   __TI_Handler_Table_Limit
0000fcf4   __TI_PINIT_Base
0000fcf8   __TI_PINIT_Limit
00011789   __TI_auto_init
080042c8   __TI_cleanup_ptr
000119fb   __TI_decompress_none
00011a09   __TI_decompress_rle24
080042cc   __TI_dtors_ptr
00000000   __TI_static_base__
000119e9   __TI_zero_init
0001181d   __aeabi_memclr
0001181d   __aeabi_memclr4
0001181d   __aeabi_memclr8
000115c1   __aeabi_memcpy
000115c1   __aeabi_memcpy4
000115c1   __aeabi_memcpy8
0001181f   __aeabi_memset
0001181f   __aeabi_memset4
0001181f   __aeabi_memset8
000118f4   __aeabi_uidivmod
ffffffff   __binit__
ffffffff   __c_args__
00010584   _c_int00
0000fbec   _coreClearAuxiliaryDataFault_
0000fc08   _coreClearAuxiliaryInstructionFault_
0000fbb4   _coreClearDataFaultAddress_
0000fb7c   _coreClearDataFault_
0000fbd0   _coreClearInstructionFaultAddress_
0000fb98   _coreClearInstructionFault_
0000fae0   _coreDisableEventBusExport_
0000fb44   _coreDisableFlashEcc_
0000fb10   _coreDisableRamEcc_
0000fac8   _coreEnableEventBusExport_
0000fb28   _coreEnableFlashEcc_
0000fb5c   _coreEnableIrqVicOffset_
0000faf8   _coreEnableRamEcc_
0000fab0   _coreEnableVfp_
0000fbe4   _coreGetAuxiliaryDataFault_
0000fc00   _coreGetAuxiliaryInstructionFault_
0000fbac   _coreGetDataFaultAddress_
0000fb74   _coreGetDataFault_
0000fbc8   _coreGetInstructionFaultAddress_
0000fb90   _coreGetInstructionFault_
0000f938   _coreInitRegisters_
0000fa44   _coreInitStackPointer_
00011148   _dabort
0000fc24   _disable_FIQ_interrupt_
0000fc2c   _disable_IRQ_interrupt_
0000fc1c   _disable_interrupt_
0000fc34   _enable_interrupt_
0000fcc4   _errata_CORTEXR4_57_
0000fcdc   _errata_CORTEXR4_66_
0000fc3c   _esmCcmErrorsClear_
0000fa90   _getCPSRValue_
0000fa98   _gotoCPUIdle_
080042c0   _lock
0000ffa4   _mpuAreRegionsSeparate_
0000ff80   _mpuDisableBackgroundRegion_
0000ff48   _mpuDisable_
0000ff68   _mpuEnableBackgroundRegion_
0000ff28   _mpuEnable_
0000ff98   _mpuGetNumberOfRegions_
0000ffc8   _mpuGetRegionBaseAddress_
0000ffe8   _mpuGetRegionPermission_
0000ffdc   _mpuGetRegionType_
0000ffb8   _mpuGetRegion_
0000fcfc   _mpuInit_
0000ffc0   _mpuSetRegionBaseAddress_
0000fff4   _mpuSetRegionSizeRegister_
0000ffd0   _mpuSetRegionTypeAndPermission_
0000ffb0   _mpuSetRegion_
000119e3   _nop
0001109c   _pmuDisableCountersGlobal_
00011084   _pmuEnableCountersGlobal_
0001111c   _pmuGetCycleCount_
00011124   _pmuGetEventCount_
00011134   _pmuGetOverflow_
00011034   _pmuInit_
000110e4   _pmuResetCounters_
000110b4   _pmuResetCycleCounter_
000110cc   _pmuResetEventCounters_
0001110c   _pmuSetCountEvent_
000110fc   _pmuStartCounters_
00011104   _pmuStopCounters_
000119db   _register_lock
000119d5   _register_unlock
080042c4   _unlock
00011995   abort
0000a084   adc1GetConfigValue
0001147c   adc1Group1Interrupt
000114c8   adc1Group2Interrupt
0000124c   adc1ParityCheck
00001314   adc2ParityCheck
00009c58   adcCalibration
0000a024   adcDisableNotification
00009fd4   adcEnableNotification
00009a28   adcGetData
0000a06c   adcGetEVTPin
000097f8   adcInit
00009c28   adcIsConversionComplete
00009bf8   adcIsFifoFull
00009e34   adcMidPointCalibration
000108ec   adcNotification
00009a00   adcResetFiFo
0000a04c   adcSetEVTPin
00009954   adcStartConversion
000099d8   adcStopConversion
ffffffff   binit
000089bc   can1GetConfigValue
000013f0   can1ParityCheck
00008b14   can2GetConfigValue
000014c8   can2ParityCheck
00001590   can3ParityCheck
0000885c   canDisableErrorNotification
0000883c   canDisableStatusChangeNotification
000088b4   canDisableloopback
000087fc   canEnableErrorNotification
0000881c   canEnableStatusChangeNotification
0000887c   canEnableloopback
00010a8c   canErrorNotification
000085a4   canFillMessageObjectData
000082cc   canGetData
000087d8   canGetErrorLevel
00008424   canGetID
000087b4   canGetLastError
00008184   canInit
000089a0   canIoRxGetBit
000088e4   canIoSetDirection
00008934   canIoSetPort
00008984   canIoTxGetBit
00008758   canIsMessageBoxValid
000086fc   canIsRxMessageArrived
000086a0   canIsTxMessagePending
00010ab4   canMessageNotification
00008504   canSendRemoteFrame
00010aa0   canStatusChangeNotification
000081d0   canTransmit
0000848c   canUpdateID
0000bc80   capGetSignal
00000030   ccmSelfCheck
000026ec   ccmr4GetConfigValue
00000918   checkB0RAMECC
00000b08   checkB1RAMECC
00001bf8   checkClockMonitor
00000cf8   checkFlashECC
00001cd4   checkFlashEEPROMECC
00001e6c   checkPLL1Slip
00001f6c   checkPLL2Slip
00002030   checkRAMAddrParity
000019b0   checkRAMECC
00002150   checkRAMUERRTest
0000079c   checkefcSelfTest
00011949   copy_in
00000234   cpuSelfTest
00000ddc   cpuSelfTestFail
00011310   crc16
00000dd4   custom_dabort
08003ce6   dataconfig1_t
00011388   delay
00002b48   disableParity
00010bbc   dmaGroupANotification
00000e8c   dmaParityCheck
08001500   draw1
08002500   draw2
08003500   drl
0000e804   dwdClearFlag
0000e738   dwdCounterEnable
0000e780   dwdGenerateSysReset
0000e7d0   dwdGetStatus
0000e814   dwdGetViolationStatus
0000e6bc   dwdInit
0000e764   dwdReset
0000e748   dwdSetPreload
0000e72c   dwwdGetCurrentDownCounter
0000e6e4   dwwdInit
0000c460   ecap1GetConfigValue
00010bd8   ecap1Interrupt
0000c4f4   ecap2GetConfigValue
00010c50   ecap2Interrupt
0000c588   ecap3GetConfigValue
00010cc8   ecap3nterrupt
0000c61c   ecap4GetConfigValue
0000c6b0   ecap5GetConfigValue
0000c744   ecap6GetConfigValue
0000c3e0   ecapClearFlag
0000c340   ecapDisableAPWMMode
0000c230   ecapDisableCapture
0000c028   ecapDisableCounterLoadOnSync
0000c38c   ecapDisableInterrupt
0000c2d4   ecapEnableAPWMmode
0000c210   ecapEnableCapture
0000bff8   ecapEnableCounterLoadOnSync
0000c364   ecapEnableInterrupt
0000c400   ecapGetCAP1
0000c418   ecapGetCAP2
0000c430   ecapGetCAP3
0000c448   ecapGetCAP4
0000c3bc   ecapGetEventStatus
0000bf68   ecapInit
00010b78   ecapNotification
0000c088   ecapSetCaptureEvent1
0000c0d4   ecapSetCaptureEvent2
0000c124   ecapSetCaptureEvent3
0000c174   ecapSetCaptureEvent4
0000c1c4   ecapSetCaptureMode
0000bfd8   ecapSetCounter
0000c04c   ecapSetEventPrescaler
0000c298   ecapSetSyncOut
0000c254   ecapStartCounter
0000c274   ecapStopCounter
0000bc40   edgeDisableNotification
0000bc04   edgeEnableNotification
0000bbd8   edgeGetCounter
00010b2c   edgeNotification
0000bbac   edgeResetCounter
00000640   efcCheck
00002654   efcGetConfigValue
00000774   efcSelfTest
000006c8   efcStuckZeroTest
00002ac0   enableParity
0000275c   errata_PBIST_4
0000dfac   esmActivateNormalOperation
0000e098   esmClearStatus
0000e0d8   esmClearStatusBuffer
0000df70   esmDisableError
0000dfe8   esmDisableInterrupt
0000df44   esmEnableError
0000dfbc   esmEnableInterrupt
0000e1f8   esmEnterSelfTest
0000df28   esmError
0000e2d0   esmGetConfigValue
0000e124   esmGetStatus
0000e198   esmGetStatusBuffer
00010a10   esmGroup1Notification
00010a20   esmGroup2Notification
00010edc   esmHighInterrupt
0000ddfc   esmInit
0000e280   esmSelfTestStatus
0000e104   esmSetCounterPreloadValue
0000e014   esmSetInterruptLevel
0000df9c   esmTriggerErrorPinReset
00003960   etpwm1GetConfigValue
00003ce8   etpwm2GetConfigValue
00003fdc   etpwm3GetConfigValue
000042bc   etpwm4GetConfigValue
0000459c   etpwm5GetConfigValue
00004884   etpwm6GetConfigValue
00004b94   etpwm7GetConfigValue
00003894   etpwmClearEventFlag
00003664   etpwmClearTripCondition
00003684   etpwmClearTripInterruptFlag
00003528   etpwmDisableChopping
000032f4   etpwmDisableCmpAShadowMode
00003354   etpwmDisableCmpBShadowMode
00003184   etpwmDisableCounterLoadOnSync
000034a8   etpwmDisableDeadband
00003858   etpwmDisableInterrupt
00003734   etpwmDisableSOCA
000037cc   etpwmDisableSOCB
000030f0   etpwmDisableTimebasePeriodShadowMode
00003634   etpwmDisableTripInterrupt
0000356c   etpwmDisableTripZoneSources
000034f4   etpwmEnableChopping
000032b8   etpwmEnableCmpAShadowMode
00003314   etpwmEnableCmpBShadowMode
00003134   etpwmEnableCounterLoadOnSync
00003454   etpwmEnableDeadBand
000038d4   etpwmEnableDigitalCompareEvents
000037ec   etpwmEnableInterrupt
000036c0   etpwmEnableSOCA
00003758   etpwmEnableSOCB
00003110   etpwmEnableTimebasePeriodShadowMode
0000360c   etpwmEnableTripInterrupt
00003544   etpwmEnableTripZoneSources
000036a0   etpwmForceTripEvent
0000387c   etpwmGetEventStatus
00002cec   etpwmInit
00010b54   etpwmNotification
00003374   etpwmSetActionQualPwmA
000033e4   etpwmSetActionQualPwmB
00003068   etpwmSetClkDiv
00003278   etpwmSetCmpA
00003298   etpwmSetCmpB
000030d0   etpwmSetCount
000031e4   etpwmSetCounterMode
000034c4   etpwmSetDeadBandDelay
00003240   etpwmSetRunMode
000031a8   etpwmSetSyncOut
000030b0   etpwmSetTimebasePeriod
0000359c   etpwmSetTripAction
00002fd4   etpwmStartTBCLK
00003020   etpwmStopTBCLK
000038b4   etpwmTriggerEvent
00003220   etpwmTriggerSWSync
00010b64   etpwmTripNotification
0001199d   exit
000022b4   fmcBus1ParityCheck
0000083c   fmcBus2Check
00000878   fmcECCcheck
0000f2b4   gioDisableNotification
0000f24c   gioEnableNotification
0000f1b4   gioGetBit
0000f31c   gioGetConfigValue
0000f1dc   gioGetPort
0001165c   gioHighLevelInterrupt
0000f054   gioInit
00010ac8   gioNotification
0000f144   gioSetBit
0000f124   gioSetDirection
0000f194   gioSetPort
0000f1f4   gioToggleBit
08003cc0   gstSPICmdStatus
080042a0   gucCmdFrameType
080042a3   gucSendDataOK
080042a4   gucSpiArmToDspSpiFault
080042a1   gucSpiRevCmpltFlag
080042a2   gucSpiRevOKFlag
0000bd8c   het1GetConfigValue
00000f38   het1ParityCheck
000010a0   het2ParityCheck
0000bd74   hetGetTimestamp
0000b674   hetInit
00010b40   hetNotification
0000bd58   hetResetTimestamp
00000fe4   htu1ParityCheck
0000119c   htu2ParityCheck
080042ac   iTimeForMotorTest
080041bc   io
080042b8   kc
080042b4   ki
080042b0   kp
0000db88   linDisableLoopback
0000dbc4   linDisableNotification
0000db54   linEnableLoopback
0000dba4   linEnableNotification
0000d924   linEnterSleep
0000dbe4   linGetConfigValue
0000dacc   linGetData
0000daac   linGetIdentifier
0000d7b4   linInit
0000da5c   linIsRxReady
0000d974   linIsTxReady
00010adc   linNotification
0000d9c4   linSend
0000d8c8   linSendHeader
0000d8f8   linSendWakupSignal
0000d8a8   linSetFunctional
0000d990   linSetLength
0000d944   linSoftwareReset
0000da78   linTxRxError
000107f4   main
00008e08   mapClocks
000115c1   memcpy
00000174   memoryInit
00010a30   memoryPort0TestFailNotification
00010a4c   memoryPort1TestFailNotification
00011825   memset
000102d8   mibspi1HighLevelInterrupt
00001664   mibspi1ParityCheck
0000176c   mibspi3ParityCheck
00001890   mibspi5ParityCheck
08003ef0   mtr
0000ad44   muxInit
000023e0   pbistFail
00002460   pbistGetConfigValue
000005a8   pbistIsTestCompleted
000005c4   pbistIsTestPassed
000005f8   pbistPortTestStatus
000004ac   pbistRun
000002cc   pbistSelfCheck
00000578   pbistStop
00008db4   periphInit
00011a10   phantomInterrupt
0000b240   pinmuxGetConfigValue
0000bb7c   pwmDisableNotification
0000bb34   pwmEnableNotification
0000ba54   pwmGetSignal
00010b14   pwmNotification
0000b79c   pwmSetDuty
0000b8d8   pwmSetSignal
0000b734   pwmStart
0000b768   pwmStop
00000000   resetEntry
000116f4   rtiCompare2Interrupt
0001173c   rtiCompare3Interrupt
0000e8c4   rtiDisableNotification
0000e89c   rtiEnableNotification
0000e8e0   rtiGetConfigValue
0000e630   rtiGetCurrentTick
0000e608   rtiGetPeriod
0000e430   rtiInit
00010970   rtiNotification
0000e57c   rtiResetCounter
0000e5e0   rtiSetPeriod
0000e524   rtiStartCounter
0000e550   rtiStopCounter
0000ef10   sciDisableLoopback
0000ef9c   sciDisableNotification
0000eedc   sciEnableLoopback
0000ef34   sciEnableNotification
0000ea64   sciInit
0000ed8c   sciIsIdleDetected
0000ed70   sciIsRxReady
0000ebf0   sciIsTxReady
0000ee04   sciReceive
0000edd8   sciReceiveByte
0000eda8   sciRxError
0000ec3c   sciSend
0000ec0c   sciSendByte
0000eb70   sciSetBaudrate
0000eb50   sciSetFunctional
00000020   selftestFailNotification
00008d74   setupFlash
00008ccc   setupPLL
00007bb4   spi1GetConfigValue
00007d44   spi4GetConfigValue
00007f24   spi5GetConfigValue
00007b3c   spiDisableLoopback
00007b88   spiDisableNotification
00007b08   spiEnableLoopback
00007b58   spiEnableNotification
0000cc70   spiEndNotification
00007458   spiGetData
00006f90   spiInit
00010af0   spiNotification
0000733c   spiReceiveData
000078b0   spiSendAndGetData
0000767c   spiSendData
0000731c   spiSetFunctional
00007774   spiTransmitAndReceiveData
00007550   spiTransmitData
000095ec   sramGetConfigValue
08003cd2   stAqctlaInit
08003cde   stDeadBandInit
000025ac   stcGetConfigValue
000001b8   stcSelfCheck
00000dd8   stcSelfCheckFail
0000902c   systemGetConfigValue
00008f30   systemInit
00008ffc   systemPowerDown
00009440   tcmflashGetConfigValue
08004070   tmr
00008d2c   trimLPO
08004290   ucRXbuffer
08003be8   ucReceiveBufferArray
08003c68   ucSendBufferArray
08004280   ucTXbuffer
0000a3c8   vimChannelMap
0000a62c   vimDisableInterrupt
0000a464   vimEnableInterrupt
0000a6d8   vimGetConfigValue
0000a2f4   vimInit
00000de0   vimParityCheck
0000fffc   vimParityErrorHandler


GLOBAL SYMBOLS: SORTED BY Symbol Address 

address    name
--------   ----
00000000   __TI_static_base__
00000000   resetEntry
00000020   selftestFailNotification
00000030   ccmSelfCheck
00000174   memoryInit
000001b8   stcSelfCheck
00000234   cpuSelfTest
000002cc   pbistSelfCheck
000004ac   pbistRun
00000578   pbistStop
000005a8   pbistIsTestCompleted
000005c4   pbistIsTestPassed
000005f8   pbistPortTestStatus
00000640   efcCheck
000006c8   efcStuckZeroTest
00000774   efcSelfTest
0000079c   checkefcSelfTest
0000083c   fmcBus2Check
00000878   fmcECCcheck
00000918   checkB0RAMECC
00000b08   checkB1RAMECC
00000cf8   checkFlashECC
00000dd4   custom_dabort
00000dd8   stcSelfCheckFail
00000ddc   cpuSelfTestFail
00000de0   vimParityCheck
00000e8c   dmaParityCheck
00000f38   het1ParityCheck
00000fe4   htu1ParityCheck
000010a0   het2ParityCheck
0000119c   htu2ParityCheck
0000124c   adc1ParityCheck
00001314   adc2ParityCheck
000013f0   can1ParityCheck
000014c8   can2ParityCheck
00001590   can3ParityCheck
00001664   mibspi1ParityCheck
0000176c   mibspi3ParityCheck
00001890   mibspi5ParityCheck
000019b0   checkRAMECC
00001bf8   checkClockMonitor
00001cd4   checkFlashEEPROMECC
00001e6c   checkPLL1Slip
00001f6c   checkPLL2Slip
00002030   checkRAMAddrParity
00002150   checkRAMUERRTest
000022b4   fmcBus1ParityCheck
000023e0   pbistFail
00002460   pbistGetConfigValue
000025ac   stcGetConfigValue
00002654   efcGetConfigValue
000026ec   ccmr4GetConfigValue
0000275c   errata_PBIST_4
00002ac0   enableParity
00002b48   disableParity
00002cec   etpwmInit
00002fd4   etpwmStartTBCLK
00003020   etpwmStopTBCLK
00003068   etpwmSetClkDiv
000030b0   etpwmSetTimebasePeriod
000030d0   etpwmSetCount
000030f0   etpwmDisableTimebasePeriodShadowMode
00003110   etpwmEnableTimebasePeriodShadowMode
00003134   etpwmEnableCounterLoadOnSync
00003184   etpwmDisableCounterLoadOnSync
000031a8   etpwmSetSyncOut
000031e4   etpwmSetCounterMode
00003220   etpwmTriggerSWSync
00003240   etpwmSetRunMode
00003278   etpwmSetCmpA
00003298   etpwmSetCmpB
000032b8   etpwmEnableCmpAShadowMode
000032f4   etpwmDisableCmpAShadowMode
00003314   etpwmEnableCmpBShadowMode
00003354   etpwmDisableCmpBShadowMode
00003374   etpwmSetActionQualPwmA
000033e4   etpwmSetActionQualPwmB
00003454   etpwmEnableDeadBand
000034a8   etpwmDisableDeadband
000034c4   etpwmSetDeadBandDelay
000034f4   etpwmEnableChopping
00003528   etpwmDisableChopping
00003544   etpwmEnableTripZoneSources
0000356c   etpwmDisableTripZoneSources
0000359c   etpwmSetTripAction
0000360c   etpwmEnableTripInterrupt
00003634   etpwmDisableTripInterrupt
00003664   etpwmClearTripCondition
00003684   etpwmClearTripInterruptFlag
000036a0   etpwmForceTripEvent
000036c0   etpwmEnableSOCA
00003734   etpwmDisableSOCA
00003758   etpwmEnableSOCB
000037cc   etpwmDisableSOCB
000037ec   etpwmEnableInterrupt
00003858   etpwmDisableInterrupt
0000387c   etpwmGetEventStatus
00003894   etpwmClearEventFlag
000038b4   etpwmTriggerEvent
000038d4   etpwmEnableDigitalCompareEvents
00003960   etpwm1GetConfigValue
00003ce8   etpwm2GetConfigValue
00003fdc   etpwm3GetConfigValue
000042bc   etpwm4GetConfigValue
0000459c   etpwm5GetConfigValue
00004884   etpwm6GetConfigValue
00004b94   etpwm7GetConfigValue
00005080   DRV_Motor_start
000050b8   DRV_Motor_stop
000050fc   ReloadCapIntOVCnt
00005128   PWM_write_CmpA
00005178   PwmInit
00005648   HandleGPTmr2PrdInt
00005678   CntrlMtrProtection
000056bc   CntrlMotorStartStop
00005b2c   ReadMotorOffsetIdc
00005d04   ClearMtrPrtctCntr
00005d18   ClearSpeedFeedback
00005d2c   CntrlAsrPi
00005e50   PiAsr
0000604c   CntrlAcrPi
0000614c   PiAcr
00006314   CalculatePWMComp
0000638c   ResetSpeedTimer
000063d0   UpdateSpeed
00006654   CheckDirection
00006904   UpdateCurrent
00006a74   ReadCapSignal
00006b28   ClearSpdToZero
00006b80   CntrlPWMOutput
00006f90   spiInit
0000731c   spiSetFunctional
0000733c   spiReceiveData
00007458   spiGetData
00007550   spiTransmitData
0000767c   spiSendData
00007774   spiTransmitAndReceiveData
000078b0   spiSendAndGetData
000079f0   SpiTxStatus
00007a7c   SpiRxStatus
00007b08   spiEnableLoopback
00007b3c   spiDisableLoopback
00007b58   spiEnableNotification
00007b88   spiDisableNotification
00007bb4   spi1GetConfigValue
00007d44   spi4GetConfigValue
00007f24   spi5GetConfigValue
00008184   canInit
000081d0   canTransmit
000082cc   canGetData
00008424   canGetID
0000848c   canUpdateID
00008504   canSendRemoteFrame
000085a4   canFillMessageObjectData
000086a0   canIsTxMessagePending
000086fc   canIsRxMessageArrived
00008758   canIsMessageBoxValid
000087b4   canGetLastError
000087d8   canGetErrorLevel
000087fc   canEnableErrorNotification
0000881c   canEnableStatusChangeNotification
0000883c   canDisableStatusChangeNotification
0000885c   canDisableErrorNotification
0000887c   canEnableloopback
000088b4   canDisableloopback
000088e4   canIoSetDirection
00008934   canIoSetPort
00008984   canIoTxGetBit
000089a0   canIoRxGetBit
000089bc   can1GetConfigValue
00008b14   can2GetConfigValue
00008ccc   setupPLL
00008d2c   trimLPO
00008d74   setupFlash
00008db4   periphInit
00008e08   mapClocks
00008f30   systemInit
00008ffc   systemPowerDown
0000902c   systemGetConfigValue
00009440   tcmflashGetConfigValue
000095ec   sramGetConfigValue
000097f8   adcInit
00009954   adcStartConversion
000099d8   adcStopConversion
00009a00   adcResetFiFo
00009a28   adcGetData
00009bf8   adcIsFifoFull
00009c28   adcIsConversionComplete
00009c58   adcCalibration
00009e34   adcMidPointCalibration
00009fd4   adcEnableNotification
0000a024   adcDisableNotification
0000a04c   adcSetEVTPin
0000a06c   adcGetEVTPin
0000a084   adc1GetConfigValue
0000a2f4   vimInit
0000a3c8   vimChannelMap
0000a464   vimEnableInterrupt
0000a62c   vimDisableInterrupt
0000a6d8   vimGetConfigValue
0000ad44   muxInit
0000b240   pinmuxGetConfigValue
0000b674   hetInit
0000b734   pwmStart
0000b768   pwmStop
0000b79c   pwmSetDuty
0000b8d8   pwmSetSignal
0000ba54   pwmGetSignal
0000bb34   pwmEnableNotification
0000bb7c   pwmDisableNotification
0000bbac   edgeResetCounter
0000bbd8   edgeGetCounter
0000bc04   edgeEnableNotification
0000bc40   edgeDisableNotification
0000bc80   capGetSignal
0000bd58   hetResetTimestamp
0000bd74   hetGetTimestamp
0000bd8c   het1GetConfigValue
0000bf68   ecapInit
0000bfd8   ecapSetCounter
0000bff8   ecapEnableCounterLoadOnSync
0000c028   ecapDisableCounterLoadOnSync
0000c04c   ecapSetEventPrescaler
0000c088   ecapSetCaptureEvent1
0000c0d4   ecapSetCaptureEvent2
0000c124   ecapSetCaptureEvent3
0000c174   ecapSetCaptureEvent4
0000c1c4   ecapSetCaptureMode
0000c210   ecapEnableCapture
0000c230   ecapDisableCapture
0000c254   ecapStartCounter
0000c274   ecapStopCounter
0000c298   ecapSetSyncOut
0000c2d4   ecapEnableAPWMmode
0000c340   ecapDisableAPWMMode
0000c364   ecapEnableInterrupt
0000c38c   ecapDisableInterrupt
0000c3bc   ecapGetEventStatus
0000c3e0   ecapClearFlag
0000c400   ecapGetCAP1
0000c418   ecapGetCAP2
0000c430   ecapGetCAP3
0000c448   ecapGetCAP4
0000c460   ecap1GetConfigValue
0000c4f4   ecap2GetConfigValue
0000c588   ecap3GetConfigValue
0000c61c   ecap4GetConfigValue
0000c6b0   ecap5GetConfigValue
0000c744   ecap6GetConfigValue
0000cba0   SPI_Process
0000cbb4   SPI_DataInit
0000cc70   spiEndNotification
0000d090   ReadInputSignal
0000d244   FilterInput00
0000d2bc   FilterInput01
0000d334   FilterInput02
0000d3ac   FilterInput04
0000d424   FilterInput13
0000d49c   FilterInput14
0000d514   FilterMntnPshBttn
0000d5d8   UpdateInputSignal
0000d6b0   ReadDoorAddress
0000d7b4   linInit
0000d8a8   linSetFunctional
0000d8c8   linSendHeader
0000d8f8   linSendWakupSignal
0000d924   linEnterSleep
0000d944   linSoftwareReset
0000d974   linIsTxReady
0000d990   linSetLength
0000d9c4   linSend
0000da5c   linIsRxReady
0000da78   linTxRxError
0000daac   linGetIdentifier
0000dacc   linGetData
0000db54   linEnableLoopback
0000db88   linDisableLoopback
0000dba4   linEnableNotification
0000dbc4   linDisableNotification
0000dbe4   linGetConfigValue
0000ddfc   esmInit
0000df28   esmError
0000df44   esmEnableError
0000df70   esmDisableError
0000df9c   esmTriggerErrorPinReset
0000dfac   esmActivateNormalOperation
0000dfbc   esmEnableInterrupt
0000dfe8   esmDisableInterrupt
0000e014   esmSetInterruptLevel
0000e098   esmClearStatus
0000e0d8   esmClearStatusBuffer
0000e104   esmSetCounterPreloadValue
0000e124   esmGetStatus
0000e198   esmGetStatusBuffer
0000e1f8   esmEnterSelfTest
0000e280   esmSelfTestStatus
0000e2d0   esmGetConfigValue
0000e430   rtiInit
0000e524   rtiStartCounter
0000e550   rtiStopCounter
0000e57c   rtiResetCounter
0000e5e0   rtiSetPeriod
0000e608   rtiGetPeriod
0000e630   rtiGetCurrentTick
0000e6bc   dwdInit
0000e6e4   dwwdInit
0000e72c   dwwdGetCurrentDownCounter
0000e738   dwdCounterEnable
0000e748   dwdSetPreload
0000e764   dwdReset
0000e780   dwdGenerateSysReset
0000e79c   IsdwdKeySequenceCorrect
0000e7d0   dwdGetStatus
0000e804   dwdClearFlag
0000e814   dwdGetViolationStatus
0000e89c   rtiEnableNotification
0000e8c4   rtiDisableNotification
0000e8e0   rtiGetConfigValue
0000ea64   sciInit
0000eb50   sciSetFunctional
0000eb70   sciSetBaudrate
0000ebf0   sciIsTxReady
0000ec0c   sciSendByte
0000ec3c   sciSend
0000ed70   sciIsRxReady
0000ed8c   sciIsIdleDetected
0000eda8   sciRxError
0000edd8   sciReceiveByte
0000ee04   sciReceive
0000eedc   sciEnableLoopback
0000ef10   sciDisableLoopback
0000ef34   sciEnableNotification
0000ef9c   sciDisableNotification
0000f054   gioInit
0000f124   gioSetDirection
0000f144   gioSetBit
0000f194   gioSetPort
0000f1b4   gioGetBit
0000f1dc   gioGetPort
0000f1f4   gioToggleBit
0000f24c   gioEnableNotification
0000f2b4   gioDisableNotification
0000f31c   gioGetConfigValue
0000f4d8   Update100msTimer
0000f580   Update10msTimer
0000f628   Update1msTimer
0000f6a4   UpdateCurrentTime
0000f8c0   UpdateMtrRttnTimer
0000f900   CnfgrWatchDogRegister
0000f904   DlyLogicTimer
0000f934   DisableDog
0000f938   _coreInitRegisters_
0000fa44   _coreInitStackPointer_
0000fa90   _getCPSRValue_
0000fa98   _gotoCPUIdle_
0000fab0   _coreEnableVfp_
0000fac8   _coreEnableEventBusExport_
0000fae0   _coreDisableEventBusExport_
0000faf8   _coreEnableRamEcc_
0000fb10   _coreDisableRamEcc_
0000fb28   _coreEnableFlashEcc_
0000fb44   _coreDisableFlashEcc_
0000fb5c   _coreEnableIrqVicOffset_
0000fb74   _coreGetDataFault_
0000fb7c   _coreClearDataFault_
0000fb90   _coreGetInstructionFault_
0000fb98   _coreClearInstructionFault_
0000fbac   _coreGetDataFaultAddress_
0000fbb4   _coreClearDataFaultAddress_
0000fbc8   _coreGetInstructionFaultAddress_
0000fbd0   _coreClearInstructionFaultAddress_
0000fbe4   _coreGetAuxiliaryDataFault_
0000fbec   _coreClearAuxiliaryDataFault_
0000fc00   _coreGetAuxiliaryInstructionFault_
0000fc08   _coreClearAuxiliaryInstructionFault_
0000fc1c   _disable_interrupt_
0000fc24   _disable_FIQ_interrupt_
0000fc2c   _disable_IRQ_interrupt_
0000fc34   _enable_interrupt_
0000fc3c   _esmCcmErrorsClear_
0000fcc4   _errata_CORTEXR4_57_
0000fcdc   _errata_CORTEXR4_66_
0000fcf4   __TI_PINIT_Base
0000fcf8   __TI_PINIT_Limit
0000fcfc   _mpuInit_
0000ff28   _mpuEnable_
0000ff48   _mpuDisable_
0000ff68   _mpuEnableBackgroundRegion_
0000ff80   _mpuDisableBackgroundRegion_
0000ff98   _mpuGetNumberOfRegions_
0000ffa4   _mpuAreRegionsSeparate_
0000ffb0   _mpuSetRegion_
0000ffb8   _mpuGetRegion_
0000ffc0   _mpuSetRegionBaseAddress_
0000ffc8   _mpuGetRegionBaseAddress_
0000ffd0   _mpuSetRegionTypeAndPermission_
0000ffdc   _mpuGetRegionType_
0000ffe8   _mpuGetRegionPermission_
0000fff4   _mpuSetRegionSizeRegister_
0000fffc   vimParityErrorHandler
000102d8   mibspi1HighLevelInterrupt
00010584   _c_int00
000107f4   main
000108ec   adcNotification
00010948   CapIntSrv
00010970   rtiNotification
00010a10   esmGroup1Notification
00010a20   esmGroup2Notification
00010a30   memoryPort0TestFailNotification
00010a4c   memoryPort1TestFailNotification
00010a8c   canErrorNotification
00010aa0   canStatusChangeNotification
00010ab4   canMessageNotification
00010ac8   gioNotification
00010adc   linNotification
00010af0   spiNotification
00010b14   pwmNotification
00010b2c   edgeNotification
00010b40   hetNotification
00010b54   etpwmNotification
00010b64   etpwmTripNotification
00010b78   ecapNotification
00010bbc   dmaGroupANotification
00010bd8   ecap1Interrupt
00010c50   ecap2Interrupt
00010cc8   ecap3nterrupt
00010d70   CntrlPID
00010edc   esmHighInterrupt
00011034   _pmuInit_
00011084   _pmuEnableCountersGlobal_
0001109c   _pmuDisableCountersGlobal_
000110b4   _pmuResetCycleCounter_
000110cc   _pmuResetEventCounters_
000110e4   _pmuResetCounters_
000110fc   _pmuStartCounters_
00011104   _pmuStopCounters_
0001110c   _pmuSetCountEvent_
0001111c   _pmuGetCycleCount_
00011124   _pmuGetEventCount_
00011134   _pmuGetOverflow_
00011148   _dabort
00011230   DrawPicture1ms
00011310   crc16
00011388   delay
000113d0   ReadMotorRawIdc
0001147c   adc1Group1Interrupt
000114c8   adc1Group2Interrupt
00011520   Drv_Init
000115c1   __aeabi_memcpy
000115c1   __aeabi_memcpy4
000115c1   __aeabi_memcpy8
000115c1   memcpy
0001165c   gioHighLevelInterrupt
000116f4   rtiCompare2Interrupt
0001173c   rtiCompare3Interrupt
00011789   __TI_auto_init
0001181d   __aeabi_memclr
0001181d   __aeabi_memclr4
0001181d   __aeabi_memclr8
0001181f   __aeabi_memset
0001181f   __aeabi_memset4
0001181f   __aeabi_memset8
00011825   memset
000118f4   __aeabi_uidivmod
00011949   copy_in
00011991   C$$EXIT
00011995   abort
0001199d   exit
000119d5   _register_unlock
000119db   _register_lock
000119e3   _nop
000119e9   __TI_zero_init
000119fb   __TI_decompress_none
00011a09   __TI_decompress_rle24
00011a10   phantomInterrupt
000122dc   __TI_Handler_Table_Base
000122e8   __TI_Handler_Table_Limit
000122f0   __TI_CINIT_Base
00012300   __TI_CINIT_Limit
08001500   draw1
08002500   draw2
08003500   drl
08003be8   ucReceiveBufferArray
08003c68   ucSendBufferArray
08003cc0   gstSPICmdStatus
08003cd2   stAqctlaInit
08003cde   stDeadBandInit
08003ce6   dataconfig1_t
08003ef0   mtr
08004070   tmr
080041bc   io
08004280   ucTXbuffer
08004290   ucRXbuffer
080042a0   gucCmdFrameType
080042a1   gucSpiRevCmpltFlag
080042a2   gucSpiRevOKFlag
080042a3   gucSendDataOK
080042a4   gucSpiArmToDspSpiFault
080042ac   iTimeForMotorTest
080042b0   kp
080042b4   ki
080042b8   kc
080042bc   T
080042c0   _lock
080042c4   _unlock
080042c8   __TI_cleanup_ptr
080042cc   __TI_dtors_ptr
ffffffff   __binit__
ffffffff   __c_args__
ffffffff   binit
UNDEFED    SHT$$INIT_ARRAY$$Base
UNDEFED    SHT$$INIT_ARRAY$$Limit

[512 symbols]
